:020000040000FA
:02000000B8291D
:06000A00820720343034AF
:1000100036345334443444342D3430342E34343470
:100020002034723465345634203465347434693481
:100030007534733420347434733465347434203438
:100040004C3445342D344334493450348207203401
:100050007334443445344C348207203473346E3462
:100060006F347434743475344234820720347334FA
:1000700065346C3464346434613450348207203421
:10008000723465346B3461346534703453348207B0
:1000900020347234653464346F3463346E344534E0
:1000A0008207203453344434443482072034743477
:1000B00069346D3473346E3461347234543482076D
:1000C0007C2887287E287C287E287C287C288728F6
:1000D00087287C287C287E287C287E2887287C28E6
:1000E000B222C000C10DC10D410840040F39C40047
:1000F0004008C10044085F28C6010800C30A43182D
:100100000800C3180800C50A0130C6000800C30370
:1001100043180800C3180800C5030130C6000800D2
:100120000830AD2083210030AD2083210800083045
:10013000AD2083210830AD20832108000030AD20A0
:1001400083210130AD20832108000030AD208321C0
:100150000730AD2083218B2108000F398600061659
:100160007F2106127F2108000F393038B600F039A0
:10017000B700B70CB70CB70CB70C37084038AE2037
:1001800036080F394038AE208B2108001230B500F8
:100190008321B50BC8280330AD2083210330AD2067
:1001A00083210330AD2083210230AD208321023032
:1001B000AD2083210830AD2083210030AD20832184
:1001C0000830AD2083210030AD2083210130AD20E7
:1001D00083210030AD2083210630AD208321003003
:1001E000AD2083210C30AD208321080006150611B7
:1001F0008613861786130030C7000030C800003011
:10020000C9000030CA000130CB0001230E300800C5
:100210009E209720A5201F30B5009321350805208A
:10022000B620B50B0D299F210030AD20832104306D
:10023000AD2083219E2008009E200430B5003508A3
:100240002620B620B50B1F2908009E200730B500D8
:1002500035082C20B620B50B282908009E20073031
:10026000B50035083520B620B50B312908009E2091
:100270000730B50035083E20B620B50B3A290800F6
:100280009E200730B50035084720B620B50B43291E
:1002900008009E200330B50035085020B620B50B6D
:1002A0004C2908009E200830B50035085520B6209E
:1002B000B50B552908000330BD001030BE00BE0B41
:1002C0005F29BD0B5D2908005030BF0005155B217B
:1002D00005115B21BF0B662905110800B2009E20A5
:1002E00064215430B6206530B6207330B6207430A7
:1002F000B6202030B6203208B6209F2164290000A5
:100300000000000008001830BA00BB00BB0B8629B3
:10031000BA0B852908000430B800B900B90B8E2942
:10032000B80B8D2908005030B8008321B80B9529EF
:100330000800BD0B0800BE0B0800BF030800083012
:10034000B5009321B50BA1290800AE21AE21AE2145
:10035000AE21AE21AE21AE21AE210800FF30CE008D
:10036000B129FF30CF00CF0BB329CE0BB129080044
:100370000030B100C30000308316031386008312DF
:100380000313203086001B3083160313850083126D
:10039000031304308500C6200821F62031306E2179
:1003A0001C21EB2132306E212521022233306E21B7
:1003B0002E21202234306E213721472235306E2104
:1003C0004021712236306E214921C02237306E2102
:1003D00052214223CD290230B1000E3086009F21E8
:1003E0000C3086009F210A3086009F21063086004F
:1003F0009F210E3086009F21003086009F21B10B87
:10040000ED2908000A30BF00FF30BD00BE00831692
:100410000313051583120313B001051AB0158519CE
:1004200030150519B0143008860099213F08031DC6
:100430000C2A8316031305118312031305110800F8
:100440000A30BF00FF30BD00BE00B0018519B015F5
:10045000051AB0143008860099213F08031D252A8B
:1004600008000830BE00BE0B332ABD0B312A08003D
:100470000430BC0005153108BD00312205113108DA
:10048000BD003122BC0B3A2ABF0B382A08003B3092
:10049000BF004430B10038224230BF003D30B100CF
:1004A00038224A30BF003630B10038224F30BF000A
:1004B0003330B10038225930BF002D30B10038221E
:1004C0006430BF002830B10038226F30BF002430C4
:1004D000B10038227630BF002230B1003822051139
:1004E00008008030C5008316031305148514831299
:1004F00003132830BF00FF30BD00BE00B222C00091
:10050000C100702046080319A62AB201B301B40144
:100510004508C40064304402031C912AB20AC40096
:100520008A2A0A304402031C982AB30AC400912A7A
:1005300001304402031C9F2AB40AC400982A9E205A
:100540003208B4203308B4203408B42006158611CC
:10055000401886158610C01886149B213F08031D7D
:10056000812A08000508C2000330C205BE220330FC
:1005700005054206031DB22A42080800832108002F
:100580000330B100061186118613C330C70037301F
:10059000C8000330C9000A30CA000130CB00012373
:1005A0000E3086048611A521CC30C7003130C8003A
:1005B0000330C9000A30CA000130CB0001230E30DD
:1005C00086040611A521D530C7002B30C8000330A2
:1005D000C9000A30CA000130CB0001230E30860466
:1005E0008610A5210030C7000030C8000030C900C7
:1005F0000030CA000130CB0001230E30B10BC52AF8
:100600000800473084000008CD000830CC00CD0C35
:10061000031C0E2B861506150611112B86110615C7
:100620000611CC0B072B840A4C300402031C032B4D
:100630008617861308001430B8008321B80B1D2BD1
:100640000800061186171B23061586131B230800B6
:10065000061186171B231B231B23061586131B233A
:1006600008001B231B231B230800282331232123DD
:100670003123212321232123312328233123312313
:10068000312308008615061586149F21352308009E
:02400E00F13F80
:00000001FF
